:1000000082C0A6C0A2C3A4C0A3C0B0C0A1C0A0C0EB
:100010009FC09EC09DC09CC04CC19AC099C08145E4
:1000200086468B479048944997609B619E62A16386
:10003000A464A765AA66AC67AE68B069B280B481F3
:10004000B682B883BA84BB84BD84FF21030A14211D
:10005000375C99FFFFFFFFFFFFFFFFFFFFFFFF0080
:100060000000000000000000050B13203557687DDC
:1000700096B4D7FF1400081400080E140004080EEC
:1000800014000305080E140004080B0E11140003DD
:1000900005080B0E1014000305080B0E10121400B7
:1000A00008000E00080E0004080E000305080E00EC
:1000B00004080E1100080E1100F3F404080E1012CB
:1000C0001400080A0C0E0F10121400080EED140094
:1000D0000203040500041400040E140004081014A4
:1000E0000004080F1114000305080B0E0004080B90
:1000F0000E00EEEDECEB140E08040004080E00EB0D
:10010000ECEDEEF3F41411241FBECFEDCDBF20E0D3
:10011000A0E6B0E001C01D92AA37B207E1F7EBE715
:10012000F0E085E5808781E08383148212828683F4
:1001300011828BE0818780E58287E1E6F0E08DEF38
:1001400087838EEF8583712C55245A94B3D019C3BD
:1001500057CF815090E0FC01E45BFF4FE491E9BD93
:10016000FC01E05AFF4F849188BD0895189525B78A
:10017000277E25BF29B7226029BF21E022BF019732
:1001800028F020E188952150E9F7F9CF089588EE0D
:1001900093E0EDCF369A3699FECF95B1809160000D
:1001A00089270895CF93C72D81E0870D8F73782E0F
:1001B000662D90E0D8D26FEF8C2F90E0CF91D3C214
:1001C000FF920F931F93CF93DF93F82E0CE710E06D
:1001D000CEE7D0E0F11005C0CE01BDD2F80180839A
:1001E00004C0F8016081CE01BED221970F5F1F4F7E
:1001F000C437D10579F7DF91CF911F910F91FF900F
:100200000895D0DF81E0DCCF811103C019BC18BC98
:1002100008959FCF0F931F93CF93C82F8B01CC23AB
:1002200061F085E096DFC801A2DF19BC18BCC801E7
:100230009EDFC8019CDFC150F2CFCF911F910F917B
:100240000895EF92FF920F931F93CF93C8E0E82E8B
:10025000F12C062F10E084E17CDFC70188DF19BC98
:1002600018BCC80184DFC150B1F7CF911F910F9125
:10027000FF90EF9008951F93CF93DF938FEA87B994
:1002800086EC86B91092600010E1C0E0D0E085E015
:1002900090E06DDF7FDFC80FD11D1150C1F7CE0197
:1002A00024E0969587952A95E1F7DF91CF911F91EC
:1002B0000895189510927A0087E790E04CD2853522
:1002C00019F0612C9EDF11C0712C872D90E043D274
:1002D000682E8F3F19F080E073DF07C0872D91E013
:1002E000970D792E803488F3F6CF20918400C09149
:1002F0007E0010917F0080917C00882319F010E02F
:10030000C0E02AE12F5F90E040E050E0A4E7B0E0D9
:10031000222379F0BD016F5F7F4FFB013197E4919C
:10032000EE2319F0962F9A1BF6CF2150AD01DB0179
:10033000EFCF092F6C2F70E0A92FB0E0E02FF0E095
:10034000112321F09D012E1B3F0B05C09F01215061
:100350003109260F371F3197E40FF51FF490265906
:100360003F4FF901F082015049F79C0F90938600AE
:10037000CC2371F0112329F0292F30E021503109CD
:1003800002C020E030E0F901E659FF4F41E0408330
:1003900027E0290F322F3150E32FE91BF0E0E15025
:1003A000FF4FE491A32FB0E0A659BF4FEC93391350
:1003B000F2CFE22FF0E0E759FF4F31E050916A00B1
:1003C0004081541330E0231B20938700362D353FA6
:1003D000E8F5452D4D30B0F4809188008F3F29F429
:1003E00080917A008093880006C081E0860D682E97
:1003F000891708F0612C809188008F5F8F7180933E
:10040000880024C030917A00309388004132C0F4D3
:1004100030918100332311F0882339F081E0860D7B
:10042000682E891798F0612C11C0862D6916D9F3B2
:10043000662019F08150682E09C02150622E06C036
:100440008111F1CF80917D00882369F3512CAB9A03
:100450008FE384BB83E187BB8CEF88BB81E083BFE4
:1004600081EA8ABD8BB780628BBF8AB785608ABFFD
:1004700085B7806285BF78948CE287B986EC86B9AF
:100480003699FECF8FEF80936000C62DC53F10F0E8
:10049000612C3CC080918800803138F4E62DF0E07A
:1004A000E659FF4FC081DC2F31C071DE80917A00A8
:1004B00080938800CCE7D0E000E010E0FF24F394C4
:1004C00081E0800F0F5F1F4F98819F3F29F4219695
:1004D00008301105A9F7E2CF6DE570E09BDEF80169
:1004E000EF59FF4F608088818F2588838ADE6FE017
:1004F00070E080E28FDE88818F258883612C81DE29
:1005000046DE80917C00882311F3C8CF4BDE10E0DB
:10051000F12C8CE2D82E96ECC92EEE24EA94CE3E35
:1005200019F463E481E204C0CD3E21F468E284E181
:1005300088DE76C0CC3E11F469E203C0CB3E19F4EC
:1005400062E581E0F5CFC33F81F404E084E101DEA0
:1005500085E090E00CDE88E0FCDD81E490E007DEE1
:100560000150A1F780ED92E05AC0C43F51F584E6F6
:1005700090E0FDDD0FDE90E0292F30E0F901E25E32
:10058000FF4FE491E81710F49E5FF6CFF901E15EAA
:10059000FF4F04916DE770E0802F829586958770FC
:1005A00039DE8EEE92E0E3DD65E070E081E032DE80
:1005B00085E694E0DCDD6DE770E0802F8F712ADE48
:1005C0000DC0CE3F71F400E0009384001ADE6AEFA4
:1005D00070E081E01FDE0F5F0A31B1F7D8DDD7DDB3
:1005E0001FC0CD3F69F58FEF809385000ADE85E05F
:1005F000B0DDCDDDCCDD84E1ACDD3DDE809385007A
:1006000000DEC5DDC4DDF9CF3699FECFE092600093
:10061000F394909185008917C8F484EF91E0A7DDE9
:1006200080917A0080938800B5DD8039A0F51F5F46
:10063000183008F474CFD53190F010E0DAE0CAE059
:100640008D2FE2DD18DED7B8C6B8DECFD93028F35B
:10065000F4E1FF1510F7E0927A00D8E0DECFD23057
:1006600030F08D2F86958695D695D80F13C019BC7E
:1006700018BC85B7877E806185BFF89485B784688C
:1006800085BF8B7F85BF85B7806285BF889585B71D
:100690008F7D85BFCD2F10E042CF112416B819BC35
:1006A00018BC87B38C7F87BBC49820E061E031E041
:1006B00040E050E0E8E0999B06C0CA010197F1F7DD
:1006C0008AB785608ABF86B38E27999B03C0511075
:1006D00003C035C0811107C090E2951590F5211136
:1006E00030C060E039E0952D71E0923208F070E0A2
:1006F000970F592E913209F4C49A611106C0211145
:1007000003C0882311F0C49821E0999885B7877EAB
:10071000806185BFA895832F887011F480E401C0A3
:1007200080E6816081BD85B7846885BF8B7F85BF8A
:1007300078948895F89481B58F7B81BDBCCF811169
:10074000D2CF8FED8DBF1FBEB5DD999A552011F028
:10075000189501C0A2DFE199FECF1FBA8EBBE09AC7
:1007600099278DB30895262FE199FECF1CBA1FBAA1
:100770008EBB2DBB0FB6F894E29AE19A0FBE01969C
:060780000895F894FFCF7C
:00000001FF
